:100C700025302E31664320202025302E3166460057
:100C80004C434420546865726D6F6D6574657200E5
:100ADB00E4FDFCC293EF7004790D8002790FE4FB07
:100AEB00C292E930E304D2918002C291D292E925FD
:100AFB00E0F90BBB04EAD291C292E4FBED25E0FDD9
:100B0B00EC33FCD292C29230910543050180035322
:100B1B0005FE0BBB0CE6D293EC540FFEEDFFAC06BF
:010B2B0022A7
:03000B00020CBB29
:060CBB00438CDC056032F1
:0C0C0600C2948F80D294C2947F327E0092
:100C1200E4FDFCC3ED9FEE6480F8EC64809850071D
:080C22000DBD00010C80EC2265
:050CC100D294C2942250
:100C9000E4FDFCD3ED9FEE6480F8EC64809850078F
:080CA0000DBD00010C80EC22E7
:07000300C295C296020C0633
:070CB400C295D296020C0666
:100BB7008B368A378938120003AB36AA37A9381221
:100BC70004D660130538E5387002053714F91204A6
:080BD700D6FF120CB480E222EB
:100B2C00C296C294758030120CC17F0A7E00120CE2
:100B3C0090120CC17F01120C90120CC1120C90750A
:100B4C008020120CC1120CC1120CC17F3812000390
:100B5C007F0C1200037F061200037F011200037F3B
:060B6C00327E00020C9035
:100A6C00055EC3E55E648094B25063E4F55E120CDF
:100A7C004EC004C005C006C007120C4EE4FBFA7948
:100A8C00107841120106E4FBFA79A0784012020FAB
:100A9C00E4FBFAF978421200158F438E428D418C9B
:100AAC0040D007D006D005D0048F3F8E3E8D3D8CB4
:100ABC003C7539FF753A0C753B707B007A007922D6
:0F0ACC001206597B007A0079227FC0120BB722E5
:100B720085585A85595B85565885575985545685E7
:100B82005557855254855355E4FF120ADB8E528F16
:100B920053E5532555CFE5523554CF2557CF35561A
:100BA200CF2559CF3558CF255BCF355AFE7C007DF6
:050BB2000512052E22D2
:100C4E00120B72AC06AD07EC1202B17B017A4D7934
:100C5E0004783D1201067B0A7AD7797978C11200A1
:020C6E0015224D
:100C2A00120B2C7BFF7A0C79807F80120BB74389D9
:100C3A0001D28CE4F560D2AFD2A9308DFDC28D12FB
:040C4A000A6C80F6BA
:10000E0002031FE86480F8E933E83360110460F0FE
:10001E00ED33EC337009E8FCE9FDEAFEEBFF220458
:10002E0060DED3EB9FEA9EE99DE8C2E78CF0C2F753
:10003E0095F0400CE8CCF8E9CDF9EACEFAEBCFFB1F
:10004E001202EA85D0F05804700320D5B3E804708C
:10005E00075002B2D502032992D5EC0460F7E4CC26
:10006E00C0E0C398F8603B94186008400DD0E0FBE8
:10007E00020301E4FBFAC9FC8028E830E406E4C977
:10008E00FBE4CAFCE830E305E4C9CACBFCE854073C
:10009E006010F8C3E913F9EA13FAEB13FBEC13FC47
:1000AE00D8F130F52FC3E49CFCEF9BFFEE9AFEEDEA
:1000BE0099FDD0E0FBEF4E4D4C701222DB03020394
:1000CE0026EC2CFCEF33FFEE33FEED33FDED30E787
:1000DE00EB020301EF2BFFEE3AFEED39FDD0E0FB14
:1000EE0050130BBB0003020329ED13FDEE13FEEFBD
:0800FE0013FFEC13FC020301E7
:10010600EC4D6011E8497017ED33EC3304600DE4F3
:10011600FCFFFEFD22E933E8330470F802031F12E8
:1001260002EA58046009E4CC2481500628500902EA
:100136000329284003020326C0E0EB4A7044B98035
:1001460006D0E0FB020315EF4E701CBD8008EBFFE6
:10015600EAFEE9FD80EBE98DF0A4FEE5F00201EF91
:10016600E9CDF9EAFEEBFFEF89F0A4FCE5F0CE89D4
:10017600F0A42EFFE435F0CD89F0A42DFEE435F091
:100186008067EF4E7005BD80D780C3EF8BF0A4ACBF
:10019600F0EE8BF0A42CFCE435F0F8EF8AF0A42CFA
:1001A600E5F038FCE433CB8DF0A42CFCE5F03BF80D
:1001B600EE8AF0A42CFCE5F038F8E433CF89F0A4FD
:1001C6002CFCE5F038CF3400CE89F0A42FFFE5F003
:1001D6003EFEE433C98DF0A42EFEE5F039CD8AF05B
:1001E600A42FFFE5F03EFEE43DFD33D0E0FB5007D3
:1001F6000BBB000F020329EC2CFCEF33FFEE33FEA2
:06020600ED33FD020301CF
:10020C00020329EC5D046005E85904700302031F26
:10021C001202EA580460F6EC4860F2EC7004FDFE41
:10022C00FF22C860DB2481C85009C39860025006C5
:10023C000203269850CAF582E9294B4A7005AB8215
:10024C0002031575F0007C1A7880C3EF9BEE9AEDD3
:10025C0099400DC3EF9BFFEE9AFEED99FDE842F03D
:10026C00DC23ACF0D0E0FFD0E0FED0E0FDAB822090
:10027C00E7101BEB60BAEC2CFCEF33FFEE33FEED1A
:10028C0033FD020301E803F830E705C0F075F00018
:10029C00EF2FFFEE33FEED33FD40B830E7C280AAFE
:1002AC0075F020800E75F010800575F0087D007ECD
:1002BC00007F003392D530D503120564EC33401027
:1002CC00EF33FFEE33FEED33FDEC33FCD5F0ED22D6
:0E02DC00E5F0247EA2D513CC92E7CDCEFF2212
:1005FD00E54D2439F8E6054D227836300702783975
:10060D00E475F0011205720204D62000EB7F2ED2A4
:10061D00008018EF540F2490D43440D4FF30040BD5
:10062D00EF24BFB41A0050032461FFE54E6002159C
:10063D004E0551E5517002055030070D7836E475C1
:10064D00F001120572EF02051C020BDF7403D207D5
:10065D008003E4C207F54D8B368A378938E4F54EB1
:10066D00F550F551E54E60077F2012063880F5757F
:10067D004FFFC201C200C202C203C205C206C208B8
:10068D00120606FF700D3007057F00120649AF51A7
:10069D00AE5022B4255FC2D5C204120606FF24D087
:1006AD00B40A00501A75F00A784E30D50508B6FF19
:1006BD000106C6A426F620D5047002D20380D924E3
:1006CD00CFB41A00EF5004C2E5D204020936D201AC
:1006DD0080C6D20080C0D20280BCD2D580BAD205ED
:1006ED0080B47F201206382002077401B54E0040F9
:1006FD00F11205FDFF120638020671D208D20680EE
:10070D00951205FDFB1205FDFA1205FDF94A4B7018
:10071D0006792D7A0A7BFF20022EE54E602A7E0097
:10072D008E827583001204EF60060EEE654F70F039
:10073D00C2D5EBC0E0EAC0E0E9C0E0EE120996D008
:10074D00E0F9D0E0FAD0E0FB1204D6FF60AAEBC0CE
:10075D00E0EAC0E0E9C0E0120638D0E02401F9D0AB
:10076D00E03400FAD0E0FBE54F0460DCD54FD980D2
:10077D0087D20280A212097960F7E54F7001041249
:10078D000334A94F600DE54F600914F54F120A208F
:10079D00EF60F3EA30E702F404C3995077EAF425E9
:1007AD004F0430E701E404F54F800D12097960C163
:1007BD00EA054F254F120334EA784CF630E701E491
:1007CD00254F04D54F0420050114120996E4C0E00D
:1007DD00120A20784CE6601320E70714F612062063
:1007ED00802204F6D0E014C0E07F00120620E54F11
:1007FD006007120617154F800B300503120617D030
:10080D00E0020671D0E00480C512097960A0E54FC1
:10081D0004120334784CEAF6E54F2005026001041A
:10082D00240412099674FF04C0E0120A2012062057
:10083D00E54F2005026003120617D0E0B54FE87FA3
:10084D004512062A784CE67F2B30E7047F2DF40401
:10085D00C0E0120638D0E075F00A84C0F01206210F
:10086D00D0E0120621020671791080027908C206C5
:10087D00C2088008D2D5790A8004790AC2D5E54F1D
:05088D00047002F54FAC
:10089200E4FAFDFEFF1205FDFC7B082001131205A0
:1008A200FDFD7B1030000A1205FDFE1205FDFF7BE7
:1008B20020EC3382D592D55013C3E43000069FFF5B
:1008C200E49EFEE42001039DFDE49CFCE4CBF8C21F
:1008D20001EC700CCFCECDCCE824F8F870F3801781
:1008E200C3EF33FFEE33FEED33FDEC33FCEB33FBB2
:1008F200994002FB0FD8E9EB300105F8D0E0C4487B
:10090200B201C0E00AEC4D4E4F78207B0070C2EA83
:10091200B54F0040BCC0E0120998D0F0D0E02001F1
:1009220004C4C0E0C4B201C0F0120621D0F0D5F078
:10093200EB020671120582070E5308755806DF4C4A
:1009420006DB4208794F08814408814906F44308CE
:10095200875507B8460816450782470A4D5006E3F1
:100962002D06E72E070A2B06EB230708200A3B2A4F
:1009720006A34800000702E54FB4FF03754F0612B5
:1009820005FDFC1205FDFD1205FDFE1205FDFF78B9
:1009920045020363790AA2D5200314300509B91070
:1009A200020404B9080104A2D52006025001042061
:1009B20002689202B54E005034C0E07F2030031925
:1009C2007F30A20272067205500F1209EFC202C2F4
:1009D20006C205C2087F30800F300503E9C0E0126D
:1009E2000638300503D0E0F9D0E0B54ECC3005171B
:1009F2007F30B9100C1206387F583004077F788098
:100A020003B908031206383002057F2D0206387F2B
:100A1200202008F87F2B2006F322920280CF7F004D
:100A2200B4070050052445F8E6FF22286E756C6C69
:100A320029002D50434958D2011205FD3001F8C258
:100A420001784E30D50108F60206A31205FD2403F3
:100A5200B405004001E4900A3493120629743A1254
:0A0A62000629D203754E0402087540
:1002EA00E9D2E7C933E833F892D5EDD2E7CD33EC5A
:0702FA0033FC5002B2D522D3
:10030100EC30E7100FBF000C0EBE00080DBD00045D
:100311000BEB6014A2D5EB13FCED92E7FD2274FF09
:10032100FCFDFEFF22E480F8A2D574FF13FC7D8062
:03033100E480EF76
:10033400F920E72824F950037907E4F42402FB1890
:10034400DBFDE624FB5014E9600DE4F618E604F640
:0F035400B40A08E4F6D9F57401F60A22C2D522DC
:10036300ED33EC3392D5FA602AB4FF33EDC2E77B69
:10037300FF60067A037988E4227A03799120D50411
:100383007A03798C224E614E002B494E46002D494B
:100393004E4600E47A08F608DAFC7B00740722E88C
:1003A300C0E0ECC0E0EDC0E0EEC0E0EFC0E0EA7515
:1003B300F010A4CAABF075F04DA42BFBE435F0FCB0
:1003C300EA2410FAEB34C5FBEC34D9FCEDC2E7FFA9
:1003D30075F056A4F42411C5F0F434C58FF0A42AA3
:1003E300E5F03BE43CF620E714120496D0E0FFD09E
:1003F300E0FED0E0FDD0E0FC12020F8014F4041202
:100403000496D0E0FFD0E0FED0E0FDD0E0FC120186
:1004130006D0E0F8E6FAEDD2E7CD33EC332482FBE5
:10042300E4C3CF33CFCE33CECD33CD33DBF37B0732
:1004330075F00A846004F6081B0AE5F0F6088FF0ED
:10044300740AA4FFACF08EF0740AA42CFEACF05036
:10045300010C8DF0740AA42CFDE435F0F608DBDE04
:03046300740722F9
:100466003F8000004120000042C80000447A00009E
:10047600461C400047C35000497424004B18968020
:100486004CBEBC205A0E1BCA6753C21C749DC5AE17
:10049600FB60065407601C23231204C4EB54386027
:1004A600091204B01204BF120106ECF8EDF9EEFAD7
:1004B600EFCB22EB1204BF80F1543803241C9004C6
:1004C60066FE93FC0EEE93FD0EEE930ECE93FF2288
:03000000020CA847
:0C0CA800787FE4F6D8FD758178020C2AF4
:1004D600BB010689828A83E0225002E722BBFE0224
:0904E600E32289828A83E4932257
:1004EF00BB010CE58229F582E5833AF583E02250C2
:1004FF0006E92582F8E622BBFE06E92582F8E2220C
:0D050F00E58229F582E5833AF583E4932225
:10051C00BB010689828A83F0225002F722BBFE01BE
:02052C00F322B8
:10052E00C2D5EC30E709B2D5E4C39DFDE49CFCEEE8
:10053E0030E715B2D5E4C39FFFE49EFE1205A8C3B3
:10054E00E49DFDE49CFC80031205A830D507C3E4AE
:06055E009FFFE49EFE2257
:0E056400C3E49FFFE49EFEE49DFDE49CFC22A8
:10057200FAE6FB0808E6F925F0F618E6CA3AF6228A
:10058200D083D082F8E4937012740193700DA3A308
:1005920093F8740193F5828883E47374029368601C
:0605A200EFA3A3A380DF1C
:100BDF00EFB40A07740D120BEA740A309811A89932
:100BEF00B8130CC2983098FDA899C298B811F63076
:070BFF0099FDC299F599224E
:1005A800BC000BBE0029EF8DF084FFADF022E4CC37
:1005B800F875F008EF2FFFEE33FEEC33FCEE9DEC00
:1005C800984005FCEE9DFE0FD5F0E9E4CEFD22ED46
:1005D800F8F5F0EE8420D21CFEADF075F008EF2F90
:1005E800FFED33FD4007985006D5F0F222C398FD81
:0505F8000FD5F0EA221E
:00000001FF
